:100000000C9469000C9486000C9486000C94860075
:100010000C9486000C9486000C9486000C94860048
:100020000C9486000C9486000C9486000C948F022D
:100030000C94B7020C9486000C9486000C948600F5
:100040000C9486000C9486000C9486000C94860018
:100050000C9486000C9486000C9486000C94860008
:100060000C9486000C9486000C9486000C948600F8
:100070000C94860012010002FF000010ADDEEEBEFF
:1000800000010102030104030904140342006C008F
:10009000750062006200460069007300680000009D
:1000A00020034800610063006B00650072002D00B2
:1000B0004A0065006F007000610072006400790002
:1000C00000000E03300030003000300030003100FE
:1000D000000011241FBECFEFD4E0DEBFCDBF11E082
:1000E000A0E0B1E0E4ECFDE002C005900D92AE337B
:1000F000B107D9F721E0AEE3B1E001C01D92A4340D
:10010000B207E1F70E949E000C94E0060C940000F8
:100110008EBD0DB407FC10C090E485B1892785B968
:100120002FEF31EE84E0215030408040E1F700C0F5
:1001300000000DB407FEF1CF8EB5089586ED84B9A9
:1001400080E185B91DBC83E58CBD8FE39CE90197F7
:10015000F1F700C000002C9880EC0E9488008FE925
:100160009FE00197F1F700C000002C9A2C9880ECDA
:100170000E9488008FE99FE00197F1F700C000001E
:100180002C9A2F9AFFCFCF93C82F8A3019F48DE085
:100190000E94C300E8ECF0E0908195FFFDCFC09392
:1001A000CE0080E090E0CF910895CF93DF93CDB75C
:1001B000DEB760970FB6F894DEBF0FBECDBF2CE060
:1001C000E5E1F1E0DE01119601900D922A95E1F74B
:1001D0001D861E861F86188AFC012081233C51F44F
:1001E0008181813049F460E1CE0101960E943D0297
:1001F00081E003C080E001C080E060960FB6F89413
:10020000DEBF0FBECDBFDF91CF910895CF93DF93B7
:10021000CDB7DEB7A0970FB6F894DEBF0FBECDBF47
:100220008130A1F440E2BE016F5F7F4F0E9418024F
:10023000882361F018A2CE0101960E94BB0640E21D
:10024000BE016F5F7F4F82E80E946002A0960FB6EA
:10025000F894DEBF0FBECDBFDF91CF9108952F92EE
:100260003F924F925F927F928F929F92AF92CF92E6
:10027000DF92EF92FF920F931F93CF93DF93282F7C
:1002800090E06CE070E00E947105FC01EB5DFE4FB8
:10029000822F90E06CE070E00E947105895D9E4FB6
:1002A00041E00F2EF9EECF2ED12CF02D0F2EFBEECC
:1002B000EF2EF12CF02DAA24A3940CEE10E06DEE9D
:1002C00070E00F2EF0EF4F2E512CF02D68949924F2
:1002D00092F8812C6894772474F8DF0120812F3FF5
:1002E00059F1E6014883E701A8822081E8012883CB
:1002F0001C019C0121503109E9012881203841F07D
:10030000203441F0203241F0203141F4372D07C034
:1003100030E405C030E303C030E201C0382DE10114
:100320002881232BEB0128832C9120FF03C0D201CD
:100330001C9202C0E20198824F5F339603964530CB
:1003400061F6EAEEF0E08EE180831082DF91CF91DA
:100350001F910F91FF90EF90DF90CF90AF909F9003
:100360008F907F905F904F903F902F900895E8EE90
:10037000F0E080818570E9F30895AF92BF92CF924B
:10038000DF92EF92FF920F931F93CF93DF93D82EBC
:10039000D62FC72FE42FF0E02E173F0710F4C22E00
:1003A00001C0C42E0E94B7010D2F1C2F6894AA24EF
:1003B000A4F80F2EF8EEEF2EF12CF02D0F2EFEEFFD
:1003C000BF2EF02DC1EFD0E02C2D80E18C1508F46C
:1003D0002A2D2223D9F0F801922FDD2011F08081FF
:1003E00001C084918883915031969111F6CF622F8C
:1003F000615070E06F5F7F4F060F171FC21AF70141
:10040000B082C11007C0203129F007C0F701B082C7
:10041000CC2019F00E94B701D7CFDF91CF911F9167
:100420000F91FF90EF90DF90CF90BF90AF90089525
:100430008093E9009091F200941708F4492F442327
:10044000D1F0362FE62FF72FA1EFB0E09C919193DA
:100450009E2F931B9417D0F39091F20091110BC033
:1004600021E030E002C0220F331F8A95E2F7EAEE66
:10047000F0E020831082842F08956623E9F0109223
:10048000E900E8EEF0E0208120FFFDCF2091F200AE
:10049000211114C0282FE82FF92FA1EFB0E081918E
:1004A0008C938E2F821B8617D0F3E8EEF0E08081CC
:1004B0008E7F808381E0089580E0089580E0089534
:1004C000CF93DF93442329F18093E900E8EEF0E035
:1004D000808180FFFDCF8091F20081111CC0962F9A
:1004E000E62FF72FA8EEB0E0C1EFD0E08C9185FFAA
:1004F00002C08081888331968E2F891B8417B0F3C8
:10050000E8EEF0E080818E7F80838FE7808381E05A
:1005100003C080E001C080E0DF91CF9108951F9279
:100520000F920FB60F9211248F93EF93FF93E1EE8A
:10053000F0E08081108283FF12C01092E90081E018
:100540008093EB001092EC0082E18093ED0088E054
:100550008093F00010923E018FEF80930E01FF9187
:10056000EF918F910F900FBE0F901F9018951F92D3
:100570000F920FB60F9211243F924F925F926F929B
:100580007F928F929F92AF92BF92CF92DF92EF9223
:10059000FF920F931F932F933F934F935F936F930C
:1005A0007F938F939F93AF93BF93EF93FF93CF93DB
:1005B000DF93CDB7DEB72A97DEBFCDBF8091F400C1
:1005C00080FF58C21092E9008091E80083FF1FC2AB
:1005D000E1EFF0E08081898380818A83208130E0AF
:1005E0003C832B834081942F80E0822B932B9C8330
:1005F0008B83208130E03E832D834081942F80E0E7
:10060000822B932B9E838D83208130E038872F832C
:100610004081942F80E0822B932B98878F8382EFE9
:100620008093E8008A81863009F030C18B819C81FB
:10063000811523E0920709F4FDC048F4811551E0CB
:10064000950789F08115924009F01CC126C08230BF
:10065000B3E09B0709F402C108F4F6C0833093406D
:1006600009F010C105C1E4E7F0E044912F8138851D
:10067000BF0180E00E94BD010CC29A2F50815F3FF4
:1006800009F49B2F490F815033968111F6CF2F5FCC
:100690003F4F2230310539F410C020E030E040E017
:1006A00014E0A1E0B0E0C9016CE070E00E947105C7
:1006B000FC01EB5DFE4F812FE0CF842F880F880F68
:1006C000880F841B0F2EFBE1EF2EF02DE80E8E2DF0
:1006D00090E00E948305082F192F89E0D8018C93A0
:1006E00082E011968C9311971296EC9212971396C2
:1006F0001C92139714968C93149781E015968C9303
:10070000159716961C92169780EC17968C93179750
:100710008AEF18968C93F80139961A86198644E068
:10072000A12C88248394F82C9A2C0F2EF9E07F2E8C
:10073000F02DBB24BA940F2EF7E0CF2EF02D0F2E04
:10074000F5E0DF2EF02D6894662461F80F2EF3E0BB
:100750005F2EF02D56C07F2DDC012C912F3F09F428
:10076000792D670F515003965111F5CF7082418357
:10077000428213826483B5821682B78210863996CC
:100780006623C1F1832F932D6CE070E00E94710508
:100790009C012A5D3E4F482CC901B9016150710985
:1007A000DB015C915F3F01F1C082D182652F6795CB
:1007B0006627679564296283513441F0503441F0D3
:1007C000513841F0503841F4562D07C05F2D05C017
:1007D0005F2D03C0562D01C0552D5383DC018C9134
:1007E000848315821682379643942D5F3F4FB5E080
:1007F0004B12D2CFA985BA851196BA87A9871297CD
:1008000071F04984342D3A84842D932D6CE070E08E
:100810000E9471058B5D9E4F542F6A2D9CCF2F81B6
:1008200038854E2DB80181E00E94BD01C8010E94AB
:100830001E062FC1E6E8F0E044912F813885BF0104
:1008400080E00E94BD0125C1EAE8F0E044912F81DB
:100850003885BF0180E00E94BD011BC1E0EAF0E0E5
:1008600044912F813885BF0180E00E94BD0111C1F4
:10087000E2ECF0E044912F813885BF0180E00E94D6
:10088000BD0107C181E28093EB0003C1853071F4A3
:100890008EEF8093E800E8EEF0E0808180FFFDCFEE
:1008A0008B819C8180688093E300F3C08930C1F420
:1008B0009981911160C08B819C81019769F481E0DD
:1008C00080933E018EEF8093E80010920E0180919C
:1008D0000E010E942F01DDC081E28093EB00D9C0A0
:1008E000883089F49981903809F057C0E8EEF0E03B
:1008F000808180FFFDCF80913E018093F1008EEFDB
:100900008093E800C6C081111CC0E8EEF0E0808151
:1009100080FFFDCF8981823859F48D81E9EEF0E0C6
:1009200080838091EB0085FB882780F9108201C0CD
:1009300080E0E1EFF0E0808310828EEF8093E800AA
:10094000A8C08B30C1F48981803211F0811155C06B
:100950008D819E818230910550F480930E018EEF3F
:100960008093E80080910E010E942F0192C081E2E5
:100970008093EB008EC08A3081F489818038E9F55C
:10098000E8EEF0E0808180FFFDCF80910E01809342
:10099000F1008EEF8093E8007CC0813011F083304D
:1009A00061F58981823049F58B819C81892B29F5FC
:1009B0008D819E818F779927382F31503430E8F41C
:1009C0003EEF3093E8008093E9002A81233021F440
:1009D00081E28093EB005DC099E19093EB0021E010
:1009E00030E0F90102C0EE0FFF1F8A95E2F7CF0158
:1009F000EAEEF0E0808310824CC0CE0101960E94A6
:100A0000D500811146C081E28093EB0042C081E2B3
:100A10008093EB002FC0F22E408150E0022E02C0E6
:100A2000559547950A94E2F740FF1BC0DB012C93D4
:100A3000D6018C9182FF13C08091F200882341F08F
:100A40006091F20070E0822F0E940601F092E900AE
:100A5000E8EEF0E089EF80838FE780831AC0D80149
:100A60009C932F5F3F4F25303105A9F681E280939B
:100A7000EB000FC021E030E0E4EFF0E069EE70E061
:100A80000F2EF8EECF2ED12CF02D0BEE10E091E2D0
:100A9000C2CF2A960FB6F894DEBF0FBECDBFDF914E
:100AA000CF91FF91EF91BF91AF919F918F917F91E6
:100AB0006F915F914F913F912F911F910F91FF90F7
:100AC000EF90DF90CF90BF90AF909F908F907F90EE
:100AD0006F905F904F903F900F900FBE0F901F90C0
:100AE00018955527002480FF02C0060E571F660F79
:100AF000771F6115710521F096958795009799F7F5
:100B0000952F802D08950F931F93CF93DF938230FD
:100B1000910510F482E090E0E0914201F0914301F0
:100B200020E030E0C0E0D0E023C040815181481790
:100B30005907A8F04817590761F4828193812097DB
:100B400019F09B838A832EC09093430180934201C6
:100B500029C02115310529F04217530710F0A901CA
:100B600002C0BE01DF0102811381EF019A01F80189
:100B70003097D9F62115310509F1281B390B24309E
:100B8000310590F412968D919C9113976115710522
:100B900021F0FB019383828304C0909343018093EF
:100BA0004201FD01329644C0FD01E20FF31F819323
:100BB0009193225031092D933C933AC020914001EA
:100BC00030914101232B41F4209111013091120108
:100BD000309341012093400120910F013091100189
:100BE0002115310541F42DB73EB7409113015091C5
:100BF0001401241B350BE0914001F0914101E217F3
:100C0000F307A0F42E1B3F0B2817390778F0AC012F
:100C10004E5F5F4F2417350748F04E0F5F1F50930C
:100C20004101409340018193919302C0E0E0F0E0E4
:100C3000CF01DF91CF911F910F910895EF92FF9215
:100C40000F931F93CF93DF93009709F48FC0DC01BC
:100C5000129713961C921E921297E0904201F09008
:100C60004301E114F10489F42D913C911197280F6F
:100C7000391F80914001909141018217930789F5B6
:100C8000B0934101A093400171C0E70120E030E042
:100C900001C0EA01CA17DB0738F44A815B819E0173
:100CA00041155105B1F722C0BC0162507109FB0129
:100CB000D383C28300811181AC01400F511F4C17B7
:100CC0005D0761F448815981400F511F4E5F5F4FAE
:100CD000518340834A815B815383428321153105CF
:100CE00029F4B0934301A093420140C0F901B383BA
:100CF000A283E90169917991C60FD71FAC17BD078F
:100D000079F4DC015E914E91460F571F4E5F5F4FA5
:100D10005183408312968D919C9113979383828384
:100D2000A0E0B0E002C0D7017C01F701828193818D
:100D30000097C9F7C701029620813181820F931F66
:100D400020914001309141012817390779F410971B
:100D500029F4109243011092420104C013961C9290
:100D60001E921297F0924101E0924001CDB7DEB79A
:100D7000E6E00C94D106DC016C9161566A3108F012
:100D8000605E6F5B6D93C1F708952A883988488843
:100D90005F846E847D848C849B84AA84B984C88497
:100DA000DF80EE80FD800C811B81AA81B981CE0F8E
:100DB000D11D0FB6F894DEBF0FBECDBFED01089573
:040DC000F894FFCFD5
:100DC4000000000200000000C30000000000FF005B
:100DD400004401200056657273696F6E20312E3015
:100DE4000000000000802002812002FF2002FF207A
:0E0DF40002C12002FF2002FF2002FF200200A9
:00000001FF
